:100000000C945F000C9489000C9489000C94890076
:100010000C9489000C9489000C9489000C9489003C
:100020000C9489000C9489000C9489000C9489002C
:100030000C9489000C9489000C9489000C9489001C
:100040000C9489000C9489000C9489000C9489000C
:100050000C9489000C9489000C9489000C948900FC
:100060000C9489000C9489000C9489000C948900EC
:100070000C9489000C9489000C9489000C948900DC
:100080000C9489000C9489000C948900E900EB0021
:10009000ED00E400EF00F100F300F500F700F900D7
:1000A000FB00FD00D804D504D2049B04CF04CC048B
:1000B000C904C604C304C004BD04DB04DE04112467
:1000C0001FBECFEFD0E4DEBFCDBF11E0A0E0B1E0B6
:1000D000E0E2FAE000E00BBF02C007900D92A2320E
:1000E000B107D9F721E0A2E2B1E001C01D92A4332B
:1000F000B207E1F710E0CFE5D0E004C02197FE01A0
:100100000E940505CE35D107C9F70E9497040C94CB
:100110000E050C94000083E391E00E94000160E072
:1001200080E391E00E9443016FEF80E391E00E9441
:10013000640160E08DE291E00E9443016FEF8DE287
:1001400091E00E9464016FEF8AE291E00E946401F5
:1001500083E291E00E943B0282E291E00E9433033D
:10016000789484B7877F84BF109260000FB6F894AC
:10017000A895809160008861809360001092600073
:100180000FBE08950FB6F894A8958091600088611D
:1001900080936000109260000FBE82E291E00E94A6
:1001A0006B03E82F98E088E10FB6F894A895809348
:1001B00060000FBE90936000A8958E2F90E0FC0128
:1001C0003197EC30F10508F00895EA5BFF4F0C948D
:1001D00005050C9483030C9494030C94B8030C94BD
:1001E000C5030C94D8030C94EB030C94F4030C9407
:1001F000FD030C9410040C9423040C943104089512
:1002000084B1806B84B926988AB18C618AB980E503
:100210008CBD81E08DBD8BB1837E8BB95A9A5B9A80
:100220005C9A08958BB1837E8BB98BB160FD10C051
:1002300090E0892B8BB98BB161FD10C090E0892BC8
:100240008BB98BB162FD10C090E0892B8BB90895FA
:1002500094E0892B8BB98BB161FFF0CF98E0892BAB
:100260008BB98BB162FFF0CF90E1892B8BB90895E8
:100270006EBD0DB407FEFDCF8EB50895FC017183F0
:100280006083428308951F93CF93DF93EC01162F71
:100290006A81888199810E94120160E48881998134
:1002A0000E94380160E0888199810E943801612FA5
:1002B000888199810E94380167E088819981DF9166
:1002C000CF911F910C9412011F93CF93DF93EC01F8
:1002D000162F6A81888199810E94120160E48881C9
:1002E00099810E94380161E0888199810E943801DA
:1002F000612F888199810E94380167E08881998106
:10030000DF91CF911F910C9412011F93CF93DF9334
:10031000EC01162F6A81888199810E94120160E4A4
:10032000888199810E94380162E1888199810E94C7
:100330003801612F888199810E94380167E08881A6
:100340009981DF91CF911F910C9412011F93CF934C
:10035000DF93EC01162F6A81888199810E94120136
:1003600060E4888199810E94380163E188819981E4
:100370000E943801612F888199810E94380167E0CD
:1003800088819981DF91CF911F910C9412011F9365
:10039000CF93DF93EC016A81888199810E941201D9
:1003A00061E4888199810E94380162E188819981A4
:1003B0000E94380160E0888199810E943801182FDD
:1003C00067E0888199810E941201812FDF91CF918E
:1003D0001F9108951F93CF93DF93EC016A81888169
:1003E00099810E94120161E4888199810E943801FB
:1003F00063E1888199810E94380160E08881998158
:100400000E943801182F67E0888199810E941201AB
:10041000812FDF91CF911F910895FC01718360833B
:10042000428308950F931F93CF93DF93EC018B01C9
:100430006A81888199810E941201B8010024660FA7
:10044000771F001C660F771F001C672F702D888197
:1004500099810E943801602F660F660F888199810B
:100460000E94380167E088819981DF91CF911F91C7
:100470000F910C94120110927C0087E880937A000F
:10048000089580917C00807E682B60937C00809131
:100490007A00806480937A0083EA91E00197F1F713
:1004A00000C0000080917A0086FDFCCF809178002A
:1004B0009091790008950F931F93CF93DF9361E09C
:1004C00080E391E00E948501C1E0D0E001E010E00E
:1004D0002FEF84E39CE0215080409040E1F700C082
:1004E0000000B8010C2E01C0660F0A94EAF780E301
:1004F00091E00E9485012196C930D10549F7DF912D
:10050000CF911F910F9108950F931F93CF93DF9376
:1005100061E08DE291E00E948501C1E0D0E001E060
:1005200010E02FEF84E39CE0215080409040E1F701
:1005300000C00000B8010C2E01C0660F0A94EAF753
:100540008DE291E00E9485012196C930D10549F7DD
:10055000DF91CF911F910F910895CF93DF93C0E06A
:10056000D0E0BE0187E291E00E94120287E893E1A9
:100570000197F1F700C000002196C11594E0D9075A
:1005800081F72FE78AE196E0215080409040E1F723
:1005900000C0000060E070E087E291E0DF91CF9161
:1005A0000C941202CF93DF93C0E0D0E0BE0184E24E
:1005B00091E00E94120287E893E10197F1F700C0F1
:1005C00000002196C11594E0D90781F72FE78AE151
:1005D00096E0215080409040E1F700C0000060E0CC
:1005E00070E084E291E0DF91CF910C9412020FB69B
:1005F000F894A895809160008861809360001092C3
:1006000060000FBE60E083E291E00E944102BC0105
:1006100087E291E00E94120261E083E291E00E9491
:100620004102BC0184E291E00E94120280E391E069
:100630000E94EA01682F80E391E00E9485018AE22E
:1006400091E00E94EA01682F8DE291E00E9485010D
:10065000D9CF0E945B020E9484020E94AD020E94D8
:10066000D2020E94F70282E08093C00088E180936A
:10067000C10086E08093C2001092C50084E180939F
:10068000C40008958091C00085FFFCCF6093C60030
:1006900008958091C00085FFFCCF6093C6008091D3
:1006A000C00085FFFCCF7093C60008958091C00004
:1006B00085FFFCCF4093C6009FEF940F442351F079
:1006C000FB0121918091C00085FFFCCF2093C600E3
:1006D0009150B8F708958091C00087FFFCCF8091BA
:1006E000C60008958091C00087FFFCCF2091C6000E
:1006F00030E09091C00097FFFCCF8091C600A90127
:10070000582BCA010895CF9382E291E00E946B03B7
:10071000C82F6FEF82E291E00E9442036C2F82E2C9
:1007200091E0CF910C94420363E082E291E00E9459
:1007300042034CE066E171E082E291E00E945603E0
:1007400049E06DE071E082E291E00E9456034CE0E6
:1007500061E071E082E291E00E9456038091000125
:10076000811101C008956FEF82E291E00C94420381
:1007700082E291E00E947203BC01660F771F680F4E
:10078000791F82E291E00C94490382E291E00E9499
:100790006B03682F80E391E00E9485018091000146
:1007A000811101C008956FEF82E291E00C94420341
:1007B00082E291E00E946B03682F8DE291E00E943B
:1007C000850180910001811101C008956FEF82E2DF
:1007D00091E00C94420380E391E00E94EA01682FCB
:1007E00082E291E00C9442038DE291E00E94EA01E2
:1007F000682F82E291E00C94420382E291E00E9431
:100800007203BC0187E291E00E9412028091000114
:10081000811101C008956FEF82E291E00C944203D0
:1008200082E291E00E947203BC0184E291E00E94A6
:10083000120280910001811101C008956FEF82E2E0
:1008400091E00C94420382E291E00E946B03682FD6
:1008500083E291E00E944102BC0182E291E00C94AB
:1008600049038F929F92AF92BF92CF92DF92EF9205
:10087000FF920F931F93CF93DF9382E291E00E9448
:100880006B03882E82E291E00E946B03982E82E235
:1008900091E00E947203EC0182E291E00E947203F7
:1008A0005C0182E291E00E9472038C016FEF82E2B0
:1008B00091E00E944203A09E6001A19ED00CB09ED8
:1008C000D00C1124CC15DD050CF5BE0187E291E0BA
:1008D0000E941202A895682D83E291E00E944102D5
:1008E0007C01692D83E291E00E9441028C01B701F5
:1008F00082E291E00E944903B80182E291E00E9405
:100900004903CA0DDB1DCC15DD05FCF26FEF82E259
:1009100091E0DF91CF911F910F91FF90EF90DF90C9
:10092000CF90BF90AF909F908F900C9442030E9405
:100930008B00D8E1C8E00FB6F894A89580916000CC
:10094000886180936000109260000FBE82E291E0A7
:100950000E946B030FB6F894A895D09360000FBE69
:10096000C0936000A89590E0FC013197EC30F10550
:1009700010F7EE5AFF4F0C9405050E942304DBCFBD
:100980000E941004D8CF0E94FD03D5CF0E94F4032B
:10099000D2CF0E94EB03CFCF0E94D803CCCF0E94CE
:1009A000C503C9CF0E94B803C6CF0E949403C3CF2A
:1009B0000E948303C0CF0E943104BDCF83E391E046
:1009C0000E94FF0042E063E371E080E391E00E9457
:1009D0003E0143E063E371E08DE291E00E943E015D
:1009E00045E063E371E08AE291E00E943E0140E06D
:1009F00063E371E087E291E00E940D0241E063E36E
:100A000071E084E291E00C940D02EE0FFF1F0024D0
:100A1000001C0BBE0790F691E02D0994F894FFCFCF
:100A200001626F617264696E666F2E680031333ADD
:100A300033333A3430004D61722032382032303155
:020A400039007B
:00000001FF
